:020000040000FA
:06000000C5EF01F0120043
:0600080032EF01F01200CE
:06002A000100A603000026
:08003000000100005400000073
:08009800D9CFE6FFE1CFD9FF4B
:1000A000020EE126936A926A070EC16E80808082FA
:1000B00080848A6A1F0EE66EAFEC01F0E552000103
:1000C000010E8E6FD9CFE1FFE552E7CFD9FF1200C5
:1000D000D9CFE6FFE1CFD9FFE652DF6A540EDF5CED
:1000E00011E2DF50EA6A000FE96E010EEA22EF50DA
:1000F00000018E1502E0808001D080908092808285
:10010000DF2AECD780EC01F0F3CF02F0F4CF03F05C
:10011000800EF35C250EF458F5E380948084000192
:100120008E1D816E8E51E8248E6F8EAF02D0010E2F
:100130008E6F000EE66EE66A99EC01F0E552E5522C
:0A014000E552E552E7CFD9FF1200A7
:06014A002A0EF66E000E05
:10015000F76E000EF86E00010900F550856F09007A
:10016000F550866F03E1856701D03DD00900F55059
:10017000806F0900F550816F0900F550826F09000A
:100180000900F550E96E0900F550EA6E0900090012
:100190000900F550836F0900F550846F09000900CC
:1001A000F6CF87F0F7CF88F0F8CF89F080C0F6FF60
:1001B00081C0F7FF82C0F8FF0001835302E184533E
:1001C00007E00900F550EE6E8307F8E28407F9D7DF
:1001D00087C0F6FF88C0F7FF89C0F8FF00018507D8
:0801E000000E865BBFD7120080
:0801E80000018C6B010E8D6F0C
:1001F000330EE66EE66A7C0EE66E52EC01F0E552D6
:10020000E552E55200018B6B1200D9CFE6FFE1CF3A
:10021000D9FFE652AE50DF6EDFAE03D000018B6B2C
:100220000DD0540E00018B5D09E28B51EA6A8C25DA
:10023000E96E8D51EA22DFCFEFFF8B2BE552E552BD
:06024000E7CFD9FF120018
:0A02460007D84CEC00F0F4EC00F0D7
:1002500068EC00F0FDD7F26AF28C9D8A9F8AD09EEE
:10026000F28E1200DACFE4FFE2CFDAFFE9CFE4FF4B
:10027000EACFE4FFE652D9CFE6FFE1CFD9FF020E85
:10028000E1269EAA02D005EC01F0D9CFE1FFE552AC
:10029000E7CFD9FFE552E5CFEAFFE5CFE9FFE5CFAC
:0402A000DAFF110070
:0C02A400D9CFE6FFE1CFD9FFAC6AAB6A0E
:1002B000FE0EDBB0AC88DBA202D0AC8CAB8CDBB426
:1002C000AC8EDBA602D0AB8801D0AB8ADBA802D013
:1002D000AC8401D0AC949E98DBAC02D09D8A01D056
:1002E0009D9A9E9ADBAE02D09D8801D09D98FC0E0F
:1002F000DB50AF6EAC8AAB8EE552E7CFD9FF120070
:10030000D9CFE6FFE1CFD9FF020EE126D650DF6E4E
:10031000010ED7CFDBFFDECF02F0DDCF03F002C04E
:10032000F3FF03C0F4FFD9CFE1FFE552E7CFD9FFD8
:020330001200B9
:0E033200D9CFE6FFE1CFD9FF020EE126FD0E86
:10034000DBCFDEFFDBCFDDFF010EDB50D76EDF50F2
:0E035000D66ED9CFE1FFE552E7CFD9FF1200FC
:02035E00D9CFF5
:10036000E6FFE1CFD9FFFE0EDB507F0BD56ED76ADB
:10037000D66AF294FE0EDBAE02D0F28A01D0F29A77
:0A038000D58EE552E7CFD9FF120039
:06038A0015EE00F025EE67
:1003900000F0F86A019CA68EA69CA5EC00F023EC68
:0603A00001F0FDD7120080
:0A03A60041417F4141007F0608300D
:1003B0007F003F2040203F0041417F4141002649CE
:1003C00049493A0041417F4141007F49494936004E
:1003D0007F40404040007F4949494100007F091962
:1003E00029460041417F4141003F2040203F007E9F
:0A03F0000A090A7E007F40404040E9
:020000040030CA
:0700000000220C0E0001803C
:00000001FF
